BL51 BANKED LINKER/LOCATER V6.22                                                        10/31/2017  16:00:21  PAGE 1


BL51 BANKED LINKER/LOCATER V6.22, INVOKED BY:
D:\KEIL_V5\C51\BIN\BL51.EXE .\obj\main.obj, .\obj\test.obj, .\obj\gui.obj, .\obj\sys.obj, .\obj\STARTUP.obj, .\obj\touch
>> .obj, .\obj\LCD.obj TO .\obj\ceshi PRINT (.\ceshi.m51) RAMSIZE (256) DISABLEWARNING (16)


MEMORY MODEL: LARGE WITH FLOATING POINT ARITHMETIC


INPUT MODULES INCLUDED:
  .\obj\main.obj (MAIN)
  .\obj\test.obj (TEST)
  .\obj\gui.obj (GUI)
  .\obj\sys.obj (SYS)
  .\obj\STARTUP.obj (?C_STARTUP)
  .\obj\touch.obj (TOUCH)
  .\obj\LCD.obj (LCD)
  D:\KEIL_V5\C51\LIB\C51FPL.LIB (?C?FPADD)
  D:\KEIL_V5\C51\LIB\C51FPL.LIB (?C?FPMUL)
  D:\KEIL_V5\C51\LIB\C51FPL.LIB (?C?FPDIV)
  D:\KEIL_V5\C51\LIB\C51FPL.LIB (?C?FPCMP)
  D:\KEIL_V5\C51\LIB\C51FPL.LIB (?C?FCAST)
  D:\KEIL_V5\C51\LIB\C51FPL.LIB (?C?CASTF)
  D:\KEIL_V5\C51\LIB\C51FPL.LIB (?C?FPGETOPN)
  D:\KEIL_V5\C51\LIB\C51L.LIB (?C_INIT)
  D:\KEIL_V5\C51\LIB\C51L.LIB (?C?CLDPTR)
  D:\KEIL_V5\C51\LIB\C51L.LIB (?C?CLDOPTR)
  D:\KEIL_V5\C51\LIB\C51L.LIB (?C?UIDIV)
  D:\KEIL_V5\C51\LIB\C51L.LIB (?C?IILDX)
  D:\KEIL_V5\C51\LIB\C51L.LIB (?C?ILDIX)
  D:\KEIL_V5\C51\LIB\C51L.LIB (?C?ISTPTR)
  D:\KEIL_V5\C51\LIB\C51L.LIB (?C?LMUL)
  D:\KEIL_V5\C51\LIB\C51L.LIB (?C?ULDIV)
  D:\KEIL_V5\C51\LIB\C51L.LIB (?C?LNEG)
  D:\KEIL_V5\C51\LIB\C51L.LIB (?C?ULCMP)
  D:\KEIL_V5\C51\LIB\C51L.LIB (?C?LSTXDATA)
  D:\KEIL_V5\C51\LIB\C51L.LIB (?C?LSTKXDATA)
  D:\KEIL_V5\C51\LIB\C51L.LIB (?C?OFFXADD)
  D:\KEIL_V5\C51\LIB\C51L.LIB (STRLEN)


LINK MAP OF MODULE:  .\obj\ceshi (MAIN)


            TYPE    BASE      LENGTH    RELOCATION   SEGMENT NAME
            -----------------------------------------------------

            * * * * * * *   D A T A   M E M O R Y   * * * * * * *
            REG     0000H     0008H     ABSOLUTE     "REG BANK 0"
            IDATA   0008H     0001H     UNIT         ?STACK

            * * * * * * *  X D A T A   M E M O R Y  * * * * * * *
            XDATA   0000H     003DH     UNIT         ?XD?TOUCH_ADJUST?TOUCH
            XDATA   003DH     003DH     UNIT         _XDATA_GROUP_
            XDATA   007AH     0024H     UNIT         ?XD?_ADS_READ_XY?TOUCH
            XDATA   009EH     0011H     UNIT         ?XD?LCD
            XDATA   00AFH     0010H     UNIT         ?XD?TOUCH
            XDATA   00BFH     000EH     UNIT         ?XD?_READ_ADS2?TOUCH
            XDATA   00CDH     000DH     UNIT         ?XD?_LCD_SHOWNUM?GUI
BL51 BANKED LINKER/LOCATER V6.22                                                      10/31/2017  16:00:21  PAGE 2


            XDATA   00DAH     000AH     UNIT         ?XD?TEST
            XDATA   00E4H     0008H     UNIT         ?XD?_READ_ADS?TOUCH
            XDATA   00ECH     0006H     UNIT         ?XD?_MYPOW?GUI
            XDATA   00F2H     0005H     UNIT         ?XD?TOUCH_TEST?TEST
            XDATA   00F7H     0005H     UNIT         ?XD?READ_TP_ONCE?TOUCH
            XDATA   00FCH     0004H     UNIT         ?XD?_DROW_TOUCH_POINT?TOUCH
            XDATA   0100H     0004H     UNIT         ?XD?_TP_DRAW_BIG_POINT?TOUCH
            XDATA   0104H     0004H     UNIT         ?XD?_LCD_CLEAR?LCD
            XDATA   0108H     0001H     UNIT         ?XD?CONVERT_POS?TOUCH

            * * * * * * *   C O D E   M E M O R Y   * * * * * * *
            CODE    0000H     0003H     ABSOLUTE     
            CODE    0003H     148EH     UNIT         ?CO?GUI
            CODE    1491H     0EA0H     UNIT         ?CO?TEST
            CODE    2331H     0AB5H     UNIT         ?PR?TOUCH_ADJUST?TOUCH
            CODE    2DE6H     0641H     UNIT         ?C?LIB_CODE
            CODE    3427H     02A1H     UNIT         ?PR?_SHOW_STR?GUI
            CODE    36C8H     0243H     UNIT         ?PR?_GUI_DRAWFONT16?GUI
            CODE    390BH     0243H     UNIT         ?PR?_GUI_DRAWFONT24?GUI
            CODE    3B4EH     0243H     UNIT         ?PR?_GUI_DRAWFONT32?GUI
            CODE    3D91H     0242H     UNIT         ?PR?TOUCH_TEST?TEST
            CODE    3FD3H     021AH     UNIT         ?PR?TEST_COLOR?TEST
            CODE    41EDH     0218H     UNIT         ?PR?_LCD_SHOWCHAR?GUI
            CODE    4405H     01F8H     UNIT         ?PR?LCD_INIT?LCD
            CODE    45FDH     01F6H     UNIT         ?PR?_GUI_CIRCLE?GUI
            CODE    47F3H     01EBH     UNIT         ?PR?_LCD_DRAWLINE?GUI
            CODE    49DEH     01E2H     UNIT         ?PR?TEST_FILLREC?TEST
            CODE    4BC0H     015BH     UNIT         ?PR?TEST_CIRCLE?TEST
            CODE    4D1BH     0157H     UNIT         ?PR?_ADS_READ_XY?TOUCH
            CODE    4E72H     013DH     UNIT         ?PR?__DRAW_CIRCLE_8?GUI
            CODE    4FAFH     0139H     UNIT         ?PR?CONVERT_POS?TOUCH
            CODE    50E8H     0131H     UNIT         ?PR?_READ_ADS2?TOUCH
            CODE    5219H     0118H     UNIT         ?PR?_DROW_TOUCH_POINT?TOUCH
            CODE    5331H     0111H     UNIT         ?PR?_LCD_SHOWNUM?GUI
            CODE    5442H     0106H     UNIT         ?PR?_LCD_FILL?GUI
            CODE    5548H     00F7H     UNIT         ?PR?_DRAWTESTPAGE?TEST
            CODE    563FH     00F6H     UNIT         ?PR?PIC_TEST?TEST
            CODE    5735H     00D3H     UNIT         ?PR?_GUI_DRAWBMP16?GUI
            CODE    5808H     00CFH     UNIT         ?PR?ENGLISH_FONT_TEST?TEST
            CODE    58D7H     00C3H     UNIT         ?PR?MAIN_TEST?TEST
            CODE    599AH     00C2H     UNIT         ?PR?_LCD_SHOWSTRING?GUI
            CODE    5A5CH     00C0H     UNIT         ?PR?CHINESE_FONT_TEST?TEST
            CODE    5B1CH     00AAH     UNIT         ?PR?_LCD_DRAWRECTANGLE?GUI
            CODE    5BC6H     0092H     UNIT         ?PR?_GUI_STRCENTER?GUI
            CODE    5C58H     008CH     UNIT         ?C_C51STARTUP
            CODE    5CE4H     0081H     UNIT         ?PR?_LCD_CLEAR?LCD
            CODE    5D65H     007BH     UNIT         ?PR?READ_TP_ONCE?TOUCH
            CODE    5DE0H     0074H     UNIT         ?PR?_TP_DRAW_BIG_POINT?TOUCH
            CODE    5E54H     0064H     UNIT         ?PR?_LCD_SETWINDOWS?LCD
            CODE    5EB8H     0063H     UNIT         ?PR?_READ_ADS?TOUCH
            CODE    5F1BH     0049H     UNIT         ?PR?_MYPOW?GUI
            CODE    5F64H     0039H     UNIT         ?PR?LCD_SETPARAM?LCD
            CODE    5F9DH     0038H     UNIT         ?CO?TOUCH
            CODE    5FD5H     0033H     UNIT         ?PR?_GUI_DRAWPOINT?GUI
            CODE    6008H     002CH     UNIT         ?C_INITSEG
            CODE    6034H     002AH     UNIT         ?PR?_LCD_DRAWPOINT?LCD
            CODE    605EH     0026H     UNIT         ?PR?_DELAY_MS?SYS
BL51 BANKED LINKER/LOCATER V6.22                                                      10/31/2017  16:00:21  PAGE 3


            CODE    6084H     0026H     UNIT         ?PR?_DELAY_US?SYS
            CODE    60AAH     0025H     UNIT         ?PR?_LCD_DRAWFILLRECTANGLE?GUI
            CODE    60CFH     0022H     UNIT         ?PR?READFROMCHARFROM7843?TOUCH
            CODE    60F1H     0020H     UNIT         ?PR?MAIN?MAIN
            CODE    6111H     001FH     UNIT         ?PR?_LCD_SETCURSOR?LCD
            CODE    6130H     001BH     UNIT         ?PR?_LCD_WR_DATA_16BIT?LCD
            CODE    614BH     001BH     UNIT         ?PR?LCD_RESET?LCD
            CODE    6166H     001AH     UNIT         ?PR?_WRITECHARTO7843?TOUCH
            CODE    6180H     0017H     UNIT         ?PR?_ADS_READ_AD?TOUCH
            CODE    6197H     0015H     UNIT         ?PR?_STRLEN?STRLEN
            CODE    61ACH     0010H     UNIT         ?PR?_LCD_WRITEREG?LCD
            CODE    61BCH     000DH     UNIT         ?PR?_LCD_WR_REG?LCD
            CODE    61C9H     000DH     UNIT         ?PR?_LCD_WR_DATA?LCD
            CODE    61D6H     000BH     UNIT         ?PR?LCD_WRITERAM_PREPARE?LCD
            CODE    61E1H     0009H     UNIT         ?PR?SPISTAR?TOUCH
            CODE    61EAH     0006H     UNIT         ?PR?TPSTATE?TOUCH



OVERLAY MAP OF MODULE:   .\obj\ceshi (MAIN)


SEGMENT                                  XDATA_GROUP
  +--> CALLED SEGMENT                  START    LENGTH
------------------------------------------------------
?C_C51STARTUP                          -----    -----
  +--> ?PR?MAIN?MAIN
  +--> ?C_INITSEG

?PR?MAIN?MAIN                          -----    -----
  +--> ?PR?LCD_INIT?LCD
  +--> ?PR?MAIN_TEST?TEST
  +--> ?PR?TEST_COLOR?TEST
  +--> ?PR?TEST_FILLREC?TEST
  +--> ?PR?TEST_CIRCLE?TEST
  +--> ?PR?ENGLISH_FONT_TEST?TEST
  +--> ?PR?CHINESE_FONT_TEST?TEST
  +--> ?PR?PIC_TEST?TEST

?PR?LCD_INIT?LCD                       -----    -----
  +--> ?PR?LCD_RESET?LCD
  +--> ?PR?_LCD_WRITEREG?LCD
  +--> ?PR?_DELAY_MS?SYS
  +--> ?PR?LCD_SETPARAM?LCD

?PR?LCD_RESET?LCD                      -----    -----
  +--> ?PR?_DELAY_MS?SYS

?PR?_LCD_WRITEREG?LCD                  -----    -----
  +--> ?PR?_LCD_WR_REG?LCD
  +--> ?PR?_LCD_WR_DATA?LCD

?PR?LCD_SETPARAM?LCD                   -----    -----
  +--> ?PR?_LCD_WRITEREG?LCD

?PR?MAIN_TEST?TEST                     -----    -----
  +--> ?CO?TEST
BL51 BANKED LINKER/LOCATER V6.22                                                      10/31/2017  16:00:21  PAGE 4


  +--> ?PR?_DRAWTESTPAGE?TEST
  +--> ?PR?_GUI_STRCENTER?GUI
  +--> ?PR?_DELAY_MS?SYS

?PR?_DRAWTESTPAGE?TEST                 003EH    0003H
  +--> ?CO?TEST
  +--> ?PR?_LCD_FILL?GUI
  +--> ?PR?_GUI_STRCENTER?GUI

?PR?_LCD_FILL?GUI                      0046H    0012H
  +--> ?PR?_LCD_SETWINDOWS?LCD
  +--> ?PR?_LCD_WR_DATA_16BIT?LCD

?PR?_LCD_SETWINDOWS?LCD                0072H    0008H
  +--> ?PR?_LCD_WRITEREG?LCD
  +--> ?PR?LCD_WRITERAM_PREPARE?LCD

?PR?LCD_WRITERAM_PREPARE?LCD           -----    -----
  +--> ?PR?_LCD_WR_REG?LCD

?PR?_GUI_STRCENTER?GUI                 0041H    000DH
  +--> ?PR?_STRLEN?STRLEN
  +--> ?PR?_SHOW_STR?GUI

?PR?_SHOW_STR?GUI                      004EH    0010H
  +--> ?PR?_LCD_SHOWCHAR?GUI
  +--> ?PR?_GUI_DRAWFONT32?GUI
  +--> ?PR?_GUI_DRAWFONT24?GUI
  +--> ?PR?_GUI_DRAWFONT16?GUI

?PR?_LCD_SHOWCHAR?GUI                  005EH    0010H
  +--> ?PR?_LCD_SETWINDOWS?LCD
  +--> ?CO?GUI
  +--> ?PR?_LCD_WR_DATA_16BIT?LCD
  +--> ?PR?_LCD_DRAWPOINT?LCD

?PR?_LCD_DRAWPOINT?LCD                 -----    -----
  +--> ?PR?_LCD_SETWINDOWS?LCD
  +--> ?PR?_LCD_WR_DATA?LCD

?PR?_GUI_DRAWFONT32?GUI                005EH    0014H
  +--> ?CO?GUI
  +--> ?PR?_LCD_SETWINDOWS?LCD
  +--> ?PR?_LCD_WR_DATA_16BIT?LCD
  +--> ?PR?_LCD_DRAWPOINT?LCD

?PR?_GUI_DRAWFONT24?GUI                005EH    0014H
  +--> ?CO?GUI
  +--> ?PR?_LCD_SETWINDOWS?LCD
  +--> ?PR?_LCD_WR_DATA_16BIT?LCD
  +--> ?PR?_LCD_DRAWPOINT?LCD

?PR?_GUI_DRAWFONT16?GUI                005EH    0014H
  +--> ?CO?GUI
  +--> ?PR?_LCD_SETWINDOWS?LCD
  +--> ?PR?_LCD_WR_DATA_16BIT?LCD
  +--> ?PR?_LCD_DRAWPOINT?LCD
BL51 BANKED LINKER/LOCATER V6.22                                                      10/31/2017  16:00:21  PAGE 5



?PR?TEST_COLOR?TEST                    -----    -----
  +--> ?CO?TEST
  +--> ?PR?_DRAWTESTPAGE?TEST
  +--> ?PR?_LCD_FILL?GUI
  +--> ?PR?_SHOW_STR?GUI
  +--> ?PR?_DELAY_MS?SYS

?PR?TEST_FILLREC?TEST                  003DH    0001H
  +--> ?CO?TEST
  +--> ?PR?_DRAWTESTPAGE?TEST
  +--> ?PR?_LCD_FILL?GUI
  +--> ?PR?_LCD_DRAWRECTANGLE?GUI
  +--> ?PR?_DELAY_MS?SYS
  +--> ?PR?_LCD_DRAWFILLRECTANGLE?GUI

?PR?_LCD_DRAWRECTANGLE?GUI             003EH    0008H
  +--> ?PR?_LCD_DRAWLINE?GUI

?PR?_LCD_DRAWLINE?GUI                  0046H    001CH
  +--> ?PR?_LCD_DRAWPOINT?LCD

?PR?_LCD_DRAWFILLRECTANGLE?GUI         003EH    0008H
  +--> ?PR?_LCD_FILL?GUI

?PR?TEST_CIRCLE?TEST                   003DH    0001H
  +--> ?CO?TEST
  +--> ?PR?_DRAWTESTPAGE?TEST
  +--> ?PR?_LCD_FILL?GUI
  +--> ?PR?_GUI_CIRCLE?GUI
  +--> ?PR?_DELAY_MS?SYS

?PR?_GUI_CIRCLE?GUI                    003EH    0012H
  +--> ?PR?__DRAW_CIRCLE_8?GUI

?PR?__DRAW_CIRCLE_8?GUI                0050H    000AH
  +--> ?PR?_GUI_DRAWPOINT?GUI

?PR?_GUI_DRAWPOINT?GUI                 005AH    0002H
  +--> ?PR?_LCD_SETCURSOR?LCD
  +--> ?PR?_LCD_WR_DATA_16BIT?LCD

?PR?_LCD_SETCURSOR?LCD                 -----    -----
  +--> ?PR?_LCD_SETWINDOWS?LCD

?PR?ENGLISH_FONT_TEST?TEST             -----    -----
  +--> ?CO?TEST
  +--> ?PR?_DRAWTESTPAGE?TEST
  +--> ?PR?_LCD_SHOWSTRING?GUI
  +--> ?PR?_DELAY_MS?SYS

?PR?_LCD_SHOWSTRING?GUI                003DH    0009H
  +--> ?PR?_LCD_SHOWCHAR?GUI

?PR?CHINESE_FONT_TEST?TEST             -----    -----
  +--> ?CO?TEST
  +--> ?PR?_DRAWTESTPAGE?TEST
BL51 BANKED LINKER/LOCATER V6.22                                                      10/31/2017  16:00:21  PAGE 6


  +--> ?PR?_SHOW_STR?GUI
  +--> ?PR?_DELAY_MS?SYS

?PR?PIC_TEST?TEST                      -----    -----
  +--> ?CO?TEST
  +--> ?PR?_DRAWTESTPAGE?TEST
  +--> ?PR?_LCD_FILL?GUI
  +--> ?PR?_GUI_DRAWBMP16?GUI
  +--> ?PR?_SHOW_STR?GUI
  +--> ?PR?_DELAY_MS?SYS

?PR?_GUI_DRAWBMP16?GUI                 003DH    000BH
  +--> ?PR?_LCD_SETWINDOWS?LCD
  +--> ?PR?_LCD_WR_DATA_16BIT?LCD



SYMBOL TABLE OF MODULE:  .\obj\ceshi (MAIN)

  VALUE           TYPE          NAME
  ----------------------------------

  -------         MODULE        MAIN
  C:0000H         SYMBOL        _ICE_DUMMY_
  D:00B2H         PUBLIC        P3M0
  D:0090H         PUBLIC        P1
  D:00B1H         PUBLIC        P3M1
  D:00B0H         PUBLIC        P3
  C:60F1H         PUBLIC        main
  -------         PROC          MAIN
  C:60F1H         LINE#         55
  C:60F1H         LINE#         56
  C:60F1H         LINE#         60
  C:60F7H         LINE#         63
  C:60FAH         LINE#         66
  C:60FAH         LINE#         67
  C:60FAH         LINE#         68
  C:60FDH         LINE#         69
  C:6100H         LINE#         70
  C:6103H         LINE#         71
  C:6106H         LINE#         72
  C:6109H         LINE#         73
  C:610CH         LINE#         74
  C:610FH         LINE#         76
  -------         ENDPROC       MAIN
  -------         ENDMOD        MAIN

  -------         MODULE        TEST
  C:0000H         SYMBOL        _ICE_DUMMY_
  D:0090H         PUBLIC        P1
  D:00B0H         PUBLIC        P3
  D:00C0H         PUBLIC        P4
  C:3FD3H         PUBLIC        Test_Color
  C:3D91H         PUBLIC        Touch_Test
  C:16B1H         PUBLIC        gImage_qq
  X:00DAH         PUBLIC        ColorTab
  C:49DEH         PUBLIC        Test_FillRec
BL51 BANKED LINKER/LOCATER V6.22                                                      10/31/2017  16:00:21  PAGE 7


  C:554EH         PUBLIC        _DrawTestPage
  C:563FH         PUBLIC        Pic_test
  C:58D7H         PUBLIC        main_test
  C:4BC0H         PUBLIC        Test_Circle
  C:5A5CH         PUBLIC        Chinese_Font_test
  C:5808H         PUBLIC        English_Font_test
  -------         PROC          L?0031
  -------         ENDPROC       L?0031
  -------         PROC          _DRAWTESTPAGE
  X:003EH         SYMBOL        str
  C:554EH         LINE#         41
  C:5559H         LINE#         42
  C:5559H         LINE#         44
  C:5579H         LINE#         46
  C:55A5H         LINE#         47
  C:55ADH         LINE#         48
  C:55E1H         LINE#         49
  C:5616H         LINE#         51
  -------         ENDPROC       _DRAWTESTPAGE
  -------         PROC          MAIN_TEST
  C:58D7H         LINE#         63
  C:58D7H         LINE#         64
  C:58D7H         LINE#         65
  C:58E0H         LINE#         67
  C:590BH         LINE#         68
  C:5936H         LINE#         69
  C:5961H         LINE#         70
  C:598CH         LINE#         71
  C:5993H         LINE#         72
  -------         ENDPROC       MAIN_TEST
  -------         PROC          TEST_COLOR
  C:3FD3H         LINE#         84
  C:3FD3H         LINE#         85
  C:3FD3H         LINE#         86
  C:3FDCH         LINE#         87
  C:4008H         LINE#         88
  C:4046H         LINE#         89
  C:406FH         LINE#         90
  C:40ADH         LINE#         91
  C:40D8H         LINE#         92
  C:4116H         LINE#         93
  C:4144H         LINE#         94
  C:4182H         LINE#         95
  C:41AFH         LINE#         96
  -------         ENDPROC       TEST_COLOR
  -------         PROC          TEST_FILLREC
  -------         DO            
  X:003DH         SYMBOL        i
  -------         ENDDO         
  C:49DEH         LINE#         110
  C:49DEH         LINE#         111
  C:49DEH         LINE#         112
  C:49E3H         LINE#         113
  C:49ECH         LINE#         114
  C:4A18H         LINE#         115
  C:4A1DH         LINE#         116
  C:4A1DH         LINE#         117
BL51 BANKED LINKER/LOCATER V6.22                                                      10/31/2017  16:00:21  PAGE 8


  C:4AA5H         LINE#         118
  C:4AC0H         LINE#         119
  C:4ACFH         LINE#         120
  C:4AD6H         LINE#         121
  C:4B02H         LINE#         122
  C:4B07H         LINE#         123
  C:4B07H         LINE#         124
  C:4B8FH         LINE#         125
  C:4BAAH         LINE#         126
  C:4BB9H         LINE#         127
  -------         ENDPROC       TEST_FILLREC
  -------         PROC          TEST_CIRCLE
  -------         DO            
  X:003DH         SYMBOL        i
  -------         ENDDO         
  C:4BC0H         LINE#         140
  C:4BC0H         LINE#         141
  C:4BC0H         LINE#         142
  C:4BC5H         LINE#         143
  C:4BCEH         LINE#         144
  C:4BFAH         LINE#         145
  C:4BFFH         LINE#         146
  C:4C6DH         LINE#         147
  C:4C74H         LINE#         148
  C:4CA0H         LINE#         149
  C:4CA5H         LINE#         150
  C:4D14H         LINE#         151
  -------         ENDPROC       TEST_CIRCLE
  -------         PROC          ENGLISH_FONT_TEST
  C:5808H         LINE#         163
  C:5808H         LINE#         164
  C:5808H         LINE#         165
  C:5811H         LINE#         166
  C:581AH         LINE#         167
  C:5822H         LINE#         168
  C:583EH         LINE#         169
  C:585DH         LINE#         170
  C:5879H         LINE#         171
  C:5895H         LINE#         172
  C:58B4H         LINE#         173
  C:58D0H         LINE#         174
  -------         ENDPROC       ENGLISH_FONT_TEST
  -------         PROC          CHINESE_FONT_TEST
  C:5A5CH         LINE#         186
  C:5A5CH         LINE#         187
  C:5A5CH         LINE#         188
  C:5A65H         LINE#         189
  C:5A8EH         LINE#         190
  C:5ABBH         LINE#         191
  C:5AE8H         LINE#         192
  C:5B15H         LINE#         193
  -------         ENDPROC       CHINESE_FONT_TEST
  -------         PROC          PIC_TEST
  C:563FH         LINE#         205
  C:563FH         LINE#         206
  C:563FH         LINE#         207
  C:5648H         LINE#         208
BL51 BANKED LINKER/LOCATER V6.22                                                      10/31/2017  16:00:21  PAGE 9


  C:5674H         LINE#         209
  C:5685H         LINE#         210
  C:56B2H         LINE#         211
  C:56C3H         LINE#         212
  C:56F0H         LINE#         213
  C:5701H         LINE#         214
  C:572EH         LINE#         215
  -------         ENDPROC       PIC_TEST
  -------         PROC          TOUCH_TEST
  -------         DO            
  X:00F2H         SYMBOL        i
  X:00F3H         SYMBOL        j
  X:00F5H         SYMBOL        colorTemp
  -------         ENDDO         
  C:3D91H         LINE#         227
  C:3D91H         LINE#         228
  C:3D91H         LINE#         229
  C:3D96H         LINE#         230
  C:3D9AH         LINE#         231
  C:3D9EH         LINE#         232
  C:3DA1H         LINE#         233
  C:3DC9H         LINE#         234
  C:3DF6H         LINE#         235
  C:3DFFH         LINE#         236
  C:3DFFH         LINE#         237
  C:3DFFH         LINE#         238
  C:3E08H         LINE#         239
  C:3E08H         LINE#         240
  C:3E34H         LINE#         241
  C:3E34H         LINE#         242
  C:3E51H         LINE#         243
  C:3E51H         LINE#         244
  C:3E54H         LINE#         245
  C:3E63H         LINE#         246
  C:3E8BH         LINE#         247
  C:3EC1H         LINE#         248
  C:3EC4H         LINE#         249
  C:3F08H         LINE#         250
  C:3F08H         LINE#         251
  C:3F63H         LINE#         252
  C:3F94H         LINE#         253
  C:3FA3H         LINE#         254
  C:3FAAH         LINE#         255
  C:3FADH         LINE#         258
  C:3FC6H         LINE#         259
  C:3FC6H         LINE#         260
  C:3FD0H         LINE#         261
  -------         ENDPROC       TOUCH_TEST
  -------         ENDMOD        TEST

  -------         MODULE        GUI
  C:0000H         SYMBOL        _ICE_DUMMY_
  C:4E90H         PUBLIC        __draw_circle_8
  D:0090H         PUBLIC        P1
  D:00B0H         PUBLIC        P3
  C:5331H         PUBLIC        _LCD_ShowNum
  C:1289H         PUBLIC        tfont32
BL51 BANKED LINKER/LOCATER V6.22                                                      10/31/2017  16:00:21  PAGE 10


  C:1083H         PUBLIC        tfont24
  C:0003H         PUBLIC        asc2_1206
  C:0A67H         PUBLIC        tfont16
  C:0477H         PUBLIC        asc2_1608
  C:45FDH         PUBLIC        _gui_circle
  C:5BC6H         PUBLIC        _Gui_StrCenter
  C:5442H         PUBLIC        _LCD_Fill
  C:3427H         PUBLIC        _Show_Str
  C:5F1BH         PUBLIC        _mypow
  C:5735H         PUBLIC        _Gui_Drawbmp16
  C:47F3H         PUBLIC        _LCD_DrawLine
  C:599AH         PUBLIC        _LCD_ShowString
  C:3B4EH         PUBLIC        _GUI_DrawFont32
  C:390BH         PUBLIC        _GUI_DrawFont24
  C:36C8H         PUBLIC        _GUI_DrawFont16
  C:41FEH         PUBLIC        _LCD_ShowChar
  C:5B1CH         PUBLIC        _LCD_DrawRectangle
  C:5FF2H         PUBLIC        _GUI_DrawPoint
  C:60AAH         PUBLIC        _LCD_DrawFillRectangle
  C:5FD8H         SYMBOL        L?0197
  C:5FD9H         SYMBOL        L?0198
  C:5FE9H         SYMBOL        L?0199
  -------         PROC          L?0196
  -------         ENDPROC       L?0196
  C:5FD8H         SYMBOL        L?0197
  C:5FD9H         SYMBOL        L?0198
  C:5FE9H         SYMBOL        L?0199
  -------         PROC          _GUI_DRAWPOINT
  D:0006H         SYMBOL        x
  D:0004H         SYMBOL        y
  X:005AH         SYMBOL        color
  C:5FF2H         LINE#         37
  C:5FFAH         LINE#         38
  C:5FFAH         LINE#         39
  C:5FFDH         LINE#         40
  -------         ENDPROC       _GUI_DRAWPOINT
  -------         PROC          _LCD_FILL
  X:0046H         SYMBOL        sx
  X:0048H         SYMBOL        sy
  D:0002H         SYMBOL        ex
  X:004CH         SYMBOL        ey
  X:004EH         SYMBOL        color
  -------         DO            
  X:0050H         SYMBOL        i
  X:0052H         SYMBOL        j
  X:0054H         SYMBOL        width
  X:0056H         SYMBOL        height
  -------         ENDDO         
  C:5442H         LINE#         56
  C:5450H         LINE#         57
  C:5450H         LINE#         59
  C:546BH         LINE#         60
  C:548CH         LINE#         61
  C:54BBH         LINE#         62
  C:54D7H         LINE#         63
  C:54D7H         LINE#         64
  C:54F3H         LINE#         65
BL51 BANKED LINKER/LOCATER V6.22                                                      10/31/2017  16:00:21  PAGE 11


  C:550EH         LINE#         66
  C:551EH         LINE#         67
  -------         ENDPROC       _LCD_FILL
  -------         PROC          _LCD_DRAWLINE
  X:0046H         SYMBOL        x1
  X:0048H         SYMBOL        y1
  D:0002H         SYMBOL        x2
  X:004CH         SYMBOL        y2
  -------         DO            
  X:004EH         SYMBOL        t
  X:0050H         SYMBOL        xerr
  X:0052H         SYMBOL        yerr
  X:0054H         SYMBOL        delta_x
  X:0056H         SYMBOL        delta_y
  X:0058H         SYMBOL        distance
  X:005AH         SYMBOL        incx
  X:005CH         SYMBOL        incy
  X:005EH         SYMBOL        uRow
  X:0060H         SYMBOL        uCol
  -------         ENDDO         
  C:47F3H         LINE#         80
  C:4801H         LINE#         81
  C:4801H         LINE#         83
  C:480CH         LINE#         86
  C:4821H         LINE#         87
  C:483CH         LINE#         88
  C:484BH         LINE#         89
  C:4851H         LINE#         90
  C:486DH         LINE#         91
  C:4879H         LINE#         92
  C:488EH         LINE#         93
  C:48AAH         LINE#         94
  C:48B6H         LINE#         95
  C:48CBH         LINE#         96
  C:48F1H         LINE#         97
  C:48F6H         LINE#         98
  C:491BH         LINE#         99
  C:491BH         LINE#         100
  C:492CH         LINE#         101
  C:4940H         LINE#         102
  C:4954H         LINE#         103
  C:4970H         LINE#         104
  C:4970H         LINE#         105
  C:497CH         LINE#         106
  C:4990H         LINE#         107
  C:4990H         LINE#         108
  C:49ACH         LINE#         109
  C:49ACH         LINE#         110
  C:49B8H         LINE#         111
  C:49CCH         LINE#         112
  C:49CCH         LINE#         113
  C:49DDH         LINE#         114
  -------         ENDPROC       _LCD_DRAWLINE
  -------         PROC          _LCD_DRAWRECTANGLE
  X:003EH         SYMBOL        x1
  X:0040H         SYMBOL        y1
  X:0042H         SYMBOL        x2
BL51 BANKED LINKER/LOCATER V6.22                                                      10/31/2017  16:00:21  PAGE 12


  X:0044H         SYMBOL        y2
  C:5B1CH         LINE#         125
  C:5B32H         LINE#         126
  C:5B32H         LINE#         127
  C:5B4EH         LINE#         128
  C:5B75H         LINE#         129
  C:5B9DH         LINE#         130
  -------         ENDPROC       _LCD_DRAWRECTANGLE
  -------         PROC          _LCD_DRAWFILLRECTANGLE
  D:0006H         SYMBOL        x1
  D:0004H         SYMBOL        y1
  D:0002H         SYMBOL        x2
  X:0044H         SYMBOL        y2
  C:60AAH         LINE#         142
  C:60AAH         LINE#         143
  C:60AAH         LINE#         144
  -------         ENDPROC       _LCD_DRAWFILLRECTANGLE
  -------         PROC          L?0200
  -------         ENDPROC       L?0200
  -------         PROC          __DRAW_CIRCLE_8
  X:0050H         SYMBOL        xc
  X:0052H         SYMBOL        yc
  X:0054H         SYMBOL        x
  X:0056H         SYMBOL        y
  X:0058H         SYMBOL        c
  C:4E90H         LINE#         159
  C:4EA8H         LINE#         160
  C:4EA8H         LINE#         161
  C:4EB0H         LINE#         163
  C:4ECBH         LINE#         165
  C:4EF6H         LINE#         167
  C:4F22H         LINE#         169
  C:4F38H         LINE#         171
  C:4F4FH         LINE#         173
  C:4F7AH         LINE#         175
  -------         ENDPROC       __DRAW_CIRCLE_8
  -------         PROC          _GUI_CIRCLE
  X:003EH         SYMBOL        xc
  X:0040H         SYMBOL        yc
  X:0042H         SYMBOL        c
  X:0044H         SYMBOL        r
  X:0046H         SYMBOL        fill
  -------         DO            
  X:0048H         SYMBOL        x
  X:004AH         SYMBOL        y
  X:004CH         SYMBOL        yi
  X:004EH         SYMBOL        d
  -------         ENDDO         
  C:45FDH         LINE#         190
  C:4611H         LINE#         191
  C:4611H         LINE#         192
  C:4628H         LINE#         194
  C:463CH         LINE#         197
  C:4649H         LINE#         198
  C:4649H         LINE#         200
  C:4668H         LINE#         201
  C:468BH         LINE#         202
BL51 BANKED LINKER/LOCATER V6.22                                                      10/31/2017  16:00:21  PAGE 13


  C:46B6H         LINE#         204
  C:46C6H         LINE#         205
  C:46E7H         LINE#         206
  C:46E9H         LINE#         207
  C:471EH         LINE#         208
  C:472CH         LINE#         209
  C:472CH         LINE#         210
  C:473DH         LINE#         211
  C:4740H         LINE#         212
  C:4740H         LINE#         213
  C:4740H         LINE#         215
  C:475FH         LINE#         216
  C:476BH         LINE#         217
  C:477BH         LINE#         218
  C:479CH         LINE#         219
  C:479EH         LINE#         220
  C:47D3H         LINE#         221
  C:47E1H         LINE#         222
  C:47E1H         LINE#         223
  C:47EFH         LINE#         224
  C:47F2H         LINE#         225
  C:47F2H         LINE#         226
  -------         ENDPROC       _GUI_CIRCLE
  C:41F9H         SYMBOL        L?0202
  -------         PROC          L?0201
  -------         ENDPROC       L?0201
  C:41F9H         SYMBOL        L?0202
  -------         PROC          _LCD_SHOWCHAR
  X:005EH         SYMBOL        x
  X:0060H         SYMBOL        y
  X:0062H         SYMBOL        fc
  X:0064H         SYMBOL        bc
  X:0066H         SYMBOL        num
  X:0067H         SYMBOL        size
  X:0068H         SYMBOL        mode
  -------         DO            
  X:0069H         SYMBOL        temp
  X:006AH         SYMBOL        pos
  X:006BH         SYMBOL        t
  X:006CH         SYMBOL        colortemp
  -------         ENDDO         
  C:41FEH         LINE#         242
  C:4216H         LINE#         243
  C:4216H         LINE#         246
  C:4225H         LINE#         248
  C:422CH         LINE#         249
  C:426AH         LINE#         250
  C:4273H         LINE#         251
  C:4273H         LINE#         253
  C:4288H         LINE#         254
  C:4288H         LINE#         255
  C:42A3H         LINE#         256
  C:42CAH         LINE#         257
  C:42DEH         LINE#         258
  C:42DEH         LINE#         259
  C:42EAH         LINE#         260
  C:42F5H         LINE#         261
BL51 BANKED LINKER/LOCATER V6.22                                                      10/31/2017  16:00:21  PAGE 14


  C:42FCH         LINE#         263
  C:4304H         LINE#         265
  C:430DH         LINE#         266
  C:430DH         LINE#         267
  C:430DH         LINE#         268
  C:4323H         LINE#         269
  C:4323H         LINE#         270
  C:433EH         LINE#         271
  C:4365H         LINE#         272
  C:437AH         LINE#         273
  C:437AH         LINE#         274
  C:4389H         LINE#         275
  C:43B4H         LINE#         276
  C:43BBH         LINE#         277
  C:43C3H         LINE#         278
  C:43CCH         LINE#         279
  C:43CCH         LINE#         280
  C:43DBH         LINE#         281
  -------         ENDPROC       _LCD_SHOWCHAR
  -------         PROC          _LCD_SHOWSTRING
  X:003DH         SYMBOL        x
  X:003FH         SYMBOL        y
  X:0041H         SYMBOL        size
  X:0042H         SYMBOL        p
  X:0045H         SYMBOL        mode
  C:599AH         LINE#         295
  C:59ABH         LINE#         296
  C:59ABH         LINE#         297
  C:59CBH         LINE#         298
  C:59CBH         LINE#         299
  C:5A03H         LINE#         301
  C:5A3AH         LINE#         302
  C:5A4EH         LINE#         303
  C:5A58H         LINE#         304
  C:5A5BH         LINE#         305
  -------         ENDPROC       _LCD_SHOWSTRING
  -------         PROC          _MYPOW
  X:00ECH         SYMBOL        m
  X:00EDH         SYMBOL        n
  -------         DO            
  X:00EEH         SYMBOL        result
  -------         ENDDO         
  C:5F1BH         LINE#         317
  C:5F23H         LINE#         318
  C:5F23H         LINE#         319
  C:5F2BH         LINE#         320
  C:5F55H         LINE#         321
  C:5F63H         LINE#         322
  -------         ENDPROC       _MYPOW
  -------         PROC          _LCD_SHOWNUM
  X:00CDH         SYMBOL        x
  X:00CFH         SYMBOL        y
  X:00D1H         SYMBOL        num
  X:00D5H         SYMBOL        len
  X:00D6H         SYMBOL        size
  -------         DO            
  X:00D7H         SYMBOL        t
BL51 BANKED LINKER/LOCATER V6.22                                                      10/31/2017  16:00:21  PAGE 15


  X:00D8H         SYMBOL        temp
  X:00D9H         SYMBOL        enshow
  -------         ENDDO         
  C:5331H         LINE#         337
  C:533FH         LINE#         338
  C:533FH         LINE#         340
  C:5344H         LINE#         341
  C:5359H         LINE#         342
  C:5359H         LINE#         343
  C:538AH         LINE#         344
  C:539DH         LINE#         345
  C:539DH         LINE#         346
  C:53A1H         LINE#         347
  C:53A1H         LINE#         348
  C:53DDH         LINE#         349
  C:53DFH         LINE#         350
  C:53E5H         LINE#         352
  C:53E5H         LINE#         353
  C:5438H         LINE#         354
  C:5441H         LINE#         355
  -------         ENDPROC       _LCD_SHOWNUM
  -------         PROC          _GUI_DRAWFONT16
  X:005EH         SYMBOL        x
  X:0060H         SYMBOL        y
  X:0062H         SYMBOL        fc
  X:0064H         SYMBOL        bc
  X:0066H         SYMBOL        s
  X:0069H         SYMBOL        mode
  -------         DO            
  X:006AH         SYMBOL        i
  X:006BH         SYMBOL        j
  X:006CH         SYMBOL        k
  X:006EH         SYMBOL        HZnum
  X:0070H         SYMBOL        x0
  -------         ENDDO         
  C:36C8H         LINE#         370
  C:36DEH         LINE#         371
  C:36DEH         LINE#         375
  C:36E6H         LINE#         376
  C:36EFH         LINE#         379
  C:370FH         LINE#         380
  C:370FH         LINE#         381
  C:375FH         LINE#         382
  C:3795H         LINE#         383
  C:379AH         LINE#         384
  C:379AH         LINE#         385
  C:37ACH         LINE#         386
  C:37ACH         LINE#         387
  C:37B2H         LINE#         388
  C:37B2H         LINE#         389
  C:37FEH         LINE#         390
  C:3809H         LINE#         391
  C:380CH         LINE#         393
  C:380CH         LINE#         394
  C:381BH         LINE#         395
  C:387AH         LINE#         396
  C:3888H         LINE#         397
BL51 BANKED LINKER/LOCATER V6.22                                                      10/31/2017  16:00:21  PAGE 16


  C:38A3H         LINE#         398
  C:38A3H         LINE#         399
  C:38A8H         LINE#         400
  C:38B6H         LINE#         401
  C:38B8H         LINE#         402
  C:38B8H         LINE#         403
  C:38B8H         LINE#         405
  C:38C1H         LINE#         407
  C:38D0H         LINE#         410
  C:38D0H         LINE#         411
  C:38D0H         LINE#         412
  C:38E1H         LINE#         414
  -------         ENDPROC       _GUI_DRAWFONT16
  -------         PROC          _GUI_DRAWFONT24
  X:005EH         SYMBOL        x
  X:0060H         SYMBOL        y
  X:0062H         SYMBOL        fc
  X:0064H         SYMBOL        bc
  X:0066H         SYMBOL        s
  X:0069H         SYMBOL        mode
  -------         DO            
  X:006AH         SYMBOL        i
  X:006BH         SYMBOL        j
  X:006CH         SYMBOL        k
  X:006EH         SYMBOL        HZnum
  X:0070H         SYMBOL        x0
  -------         ENDDO         
  C:390BH         LINE#         430
  C:3921H         LINE#         431
  C:3921H         LINE#         435
  C:3929H         LINE#         436
  C:3932H         LINE#         438
  C:3952H         LINE#         439
  C:3952H         LINE#         440
  C:39A2H         LINE#         441
  C:39D8H         LINE#         442
  C:39DDH         LINE#         443
  C:39DDH         LINE#         444
  C:39EFH         LINE#         445
  C:39EFH         LINE#         446
  C:39F5H         LINE#         447
  C:39F5H         LINE#         448
  C:3A41H         LINE#         449
  C:3A4CH         LINE#         450
  C:3A4FH         LINE#         452
  C:3A4FH         LINE#         453
  C:3A5EH         LINE#         454
  C:3ABDH         LINE#         455
  C:3ACBH         LINE#         456
  C:3AE6H         LINE#         457
  C:3AE6H         LINE#         458
  C:3AEBH         LINE#         459
  C:3AF9H         LINE#         460
  C:3AFBH         LINE#         461
  C:3AFBH         LINE#         462
  C:3AFBH         LINE#         463
  C:3B04H         LINE#         464
BL51 BANKED LINKER/LOCATER V6.22                                                      10/31/2017  16:00:21  PAGE 17


  C:3B13H         LINE#         467
  C:3B13H         LINE#         468
  C:3B13H         LINE#         469
  C:3B24H         LINE#         471
  -------         ENDPROC       _GUI_DRAWFONT24
  -------         PROC          _GUI_DRAWFONT32
  X:005EH         SYMBOL        x
  X:0060H         SYMBOL        y
  X:0062H         SYMBOL        fc
  X:0064H         SYMBOL        bc
  X:0066H         SYMBOL        s
  X:0069H         SYMBOL        mode
  -------         DO            
  X:006AH         SYMBOL        i
  X:006BH         SYMBOL        j
  X:006CH         SYMBOL        k
  X:006EH         SYMBOL        HZnum
  X:0070H         SYMBOL        x0
  -------         ENDDO         
  C:3B4EH         LINE#         487
  C:3B64H         LINE#         488
  C:3B64H         LINE#         492
  C:3B6CH         LINE#         493
  C:3B75H         LINE#         494
  C:3B95H         LINE#         495
  C:3B95H         LINE#         496
  C:3BE5H         LINE#         497
  C:3C1BH         LINE#         498
  C:3C20H         LINE#         499
  C:3C20H         LINE#         500
  C:3C32H         LINE#         501
  C:3C32H         LINE#         502
  C:3C38H         LINE#         503
  C:3C38H         LINE#         504
  C:3C84H         LINE#         505
  C:3C8FH         LINE#         506
  C:3C92H         LINE#         508
  C:3C92H         LINE#         509
  C:3CA1H         LINE#         510
  C:3D00H         LINE#         511
  C:3D0EH         LINE#         512
  C:3D29H         LINE#         513
  C:3D29H         LINE#         514
  C:3D2EH         LINE#         515
  C:3D3CH         LINE#         516
  C:3D3EH         LINE#         517
  C:3D3EH         LINE#         518
  C:3D3EH         LINE#         519
  C:3D47H         LINE#         520
  C:3D56H         LINE#         523
  C:3D56H         LINE#         524
  C:3D56H         LINE#         525
  C:3D67H         LINE#         527
  -------         ENDPROC       _GUI_DRAWFONT32
  -------         PROC          _SHOW_STR
  X:004EH         SYMBOL        x
  X:0050H         SYMBOL        y
BL51 BANKED LINKER/LOCATER V6.22                                                      10/31/2017  16:00:21  PAGE 18


  X:0052H         SYMBOL        fc
  X:0054H         SYMBOL        bc
  X:0056H         SYMBOL        str
  X:0059H         SYMBOL        size
  X:005AH         SYMBOL        mode
  -------         DO            
  X:005BH         SYMBOL        x0
  X:005DH         SYMBOL        bHz
  -------         ENDDO         
  C:3427H         LINE#         544
  C:343DH         LINE#         545
  C:343DH         LINE#         546
  C:3445H         LINE#         547
  C:3448H         LINE#         548
  C:345BH         LINE#         549
  C:345BH         LINE#         550
  C:3464H         LINE#         551
  C:3464H         LINE#         552
  C:34A9H         LINE#         554
  C:34C5H         LINE#         556
  C:34C5H         LINE#         557
  C:34C9H         LINE#         558
  C:34C9H         LINE#         559
  C:34DBH         LINE#         560
  C:34EAH         LINE#         561
  C:34F4H         LINE#         562
  C:34F7H         LINE#         564
  C:34F7H         LINE#         565
  C:3508H         LINE#         566
  C:3508H         LINE#         567
  C:352FH         LINE#         568
  C:3535H         LINE#         569
  C:3537H         LINE#         571
  C:3537H         LINE#         572
  C:3568H         LINE#         573
  C:357CH         LINE#         574
  C:357CH         LINE#         575
  C:357CH         LINE#         576
  C:3586H         LINE#         578
  C:3586H         LINE#         579
  C:3589H         LINE#         580
  C:3589H         LINE#         581
  C:35CCH         LINE#         583
  C:35D1H         LINE#         584
  C:35D5H         LINE#         585
  C:3617H         LINE#         586
  C:3622H         LINE#         587
  C:3666H         LINE#         589
  C:36A8H         LINE#         591
  C:36B2H         LINE#         592
  C:36C4H         LINE#         593
  C:36C4H         LINE#         594
  C:36C7H         LINE#         595
  -------         ENDPROC       _SHOW_STR
  -------         PROC          _GUI_STRCENTER
  X:0041H         SYMBOL        x
  X:0043H         SYMBOL        y
BL51 BANKED LINKER/LOCATER V6.22                                                      10/31/2017  16:00:21  PAGE 19


  X:0045H         SYMBOL        fc
  X:0047H         SYMBOL        bc
  X:0049H         SYMBOL        str
  X:004CH         SYMBOL        size
  X:004DH         SYMBOL        mode
  -------         DO            
  D:0006H         SYMBOL        len
  D:0006H         SYMBOL        x1
  -------         ENDDO         
  C:5BC6H         LINE#         611
  C:5BDAH         LINE#         612
  C:5BDAH         LINE#         613
  C:5BE8H         LINE#         614
  C:5C05H         LINE#         615
  -------         ENDPROC       _GUI_STRCENTER
  -------         PROC          _GUI_DRAWBMP16
  X:003DH         SYMBOL        x
  X:003FH         SYMBOL        y
  X:0041H         SYMBOL        p
  -------         DO            
  X:0044H         SYMBOL        i
  X:0046H         SYMBOL        picH
  X:0047H         SYMBOL        picL
  -------         ENDDO         
  C:5735H         LINE#         628
  C:5750H         LINE#         629
  C:5750H         LINE#         632
  C:577CH         LINE#         633
  C:5783H         LINE#         634
  C:5783H         LINE#         635
  C:57A6H         LINE#         636
  C:57B6H         LINE#         637
  C:57BFH         LINE#         638
  C:57DEH         LINE#         639
  -------         ENDPROC       _GUI_DRAWBMP16
  -------         ENDMOD        GUI

  -------         MODULE        SYS
  C:0000H         SYMBOL        _ICE_DUMMY_
  C:605EH         PUBLIC        _delay_ms
  C:6084H         PUBLIC        _delay_us
  -------         PROC          _DELAY_MS
  D:0006H         SYMBOL        count
  -------         DO            
  D:0004H         SYMBOL        i
  D:0002H         SYMBOL        j
  -------         ENDDO         
  C:605EH         LINE#         2
  C:605EH         LINE#         3
  C:605EH         LINE#         5
  C:606EH         LINE#         6
  C:6083H         LINE#         7
  -------         ENDPROC       _DELAY_MS
  -------         PROC          _DELAY_US
  D:0006H         SYMBOL        count
  -------         DO            
  D:0004H         SYMBOL        i
BL51 BANKED LINKER/LOCATER V6.22                                                      10/31/2017  16:00:21  PAGE 20


  D:0002H         SYMBOL        j
  -------         ENDDO         
  C:6084H         LINE#         9
  C:6084H         LINE#         10
  C:6084H         LINE#         12
  C:6094H         LINE#         13
  C:60A9H         LINE#         14
  -------         ENDPROC       _DELAY_US
  -------         ENDMOD        SYS

  -------         MODULE        ?C_STARTUP
  C:5C58H         SEGMENT       ?C_C51STARTUP
  I:0008H         SEGMENT       ?STACK
  C:0000H         PUBLIC        ?C_STARTUP
  D:00E0H         SYMBOL        ACC
  D:00F0H         SYMBOL        B
  D:0083H         SYMBOL        DPH
  D:0082H         SYMBOL        DPL
  N:0000H         SYMBOL        IBPSTACK
  N:0100H         SYMBOL        IBPSTACKTOP
  N:0080H         SYMBOL        IDATALEN
  C:5C5BH         SYMBOL        IDATALOOP
  N:0000H         SYMBOL        PBPSTACK
  N:0100H         SYMBOL        PBPSTACKTOP
  N:0000H         SYMBOL        PDATALEN
  N:0000H         SYMBOL        PDATASTART
  N:0000H         SYMBOL        PPAGE
  N:0000H         SYMBOL        PPAGEENABLE
  D:00A0H         SYMBOL        PPAGE_SFR
  D:0081H         SYMBOL        SP
  C:5C58H         SYMBOL        STARTUP1
  N:0000H         SYMBOL        XBPSTACK
  N:0000H         SYMBOL        XBPSTACKTOP
  N:0000H         SYMBOL        XDATALEN
  N:0000H         SYMBOL        XDATASTART
  C:0000H         LINE#         126
  C:5C58H         LINE#         133
  C:5C5AH         LINE#         134
  C:5C5BH         LINE#         135
  C:5C5CH         LINE#         136
  C:5C5EH         LINE#         185
  C:5C61H         LINE#         196
  -------         ENDMOD        ?C_STARTUP

  -------         MODULE        TOUCH
  C:0000H         SYMBOL        _ICE_DUMMY_
  D:0090H         PUBLIC        P1
  D:00B0H         PUBLIC        P3
  D:00C0H         PUBLIC        P4
  C:60CFH         PUBLIC        ReadFromCharFrom7843
  C:61EAH         PUBLIC        tpstate
  C:61E1H         PUBLIC        spistar
  B:00D0H.7       PUBLIC        CY
  C:6180H         PUBLIC        _ADS_Read_AD
  B:00B0H.6       PUBLIC        DCLK
  C:6166H         PUBLIC        _WriteCharTo7843
  C:5EB8H         PUBLIC        _Read_ADS
BL51 BANKED LINKER/LOCATER V6.22                                                      10/31/2017  16:00:21  PAGE 21


  B:00B0H.5       PUBLIC        DOUT
  X:00AFH         PUBLIC        chx
  X:00B1H         PUBLIC        chy
  C:4D1BH         PUBLIC        _ADS_Read_XY
  X:00B3H         PUBLIC        tp_pixlcd
  C:2331H         PUBLIC        Touch_Adjust
  B:00B0H.4       PUBLIC        DIN
  X:00B7H         PUBLIC        tp_pixad
  C:50E8H         PUBLIC        _Read_ADS2
  C:5D65H         PUBLIC        Read_TP_Once
  B:00B0H.7       PUBLIC        TCS
  X:00BBH         PUBLIC        vx
  X:00BDH         PUBLIC        vy
  C:5219H         PUBLIC        _Drow_Touch_Point
  B:00C0H.0       PUBLIC        Penirq
  C:5DE0H         PUBLIC        _TP_Draw_Big_Point
  C:4FAFH         PUBLIC        Convert_Pos
  -------         PROC          TPSTATE
  C:61EAH         LINE#         14
  C:61EAH         LINE#         15
  C:61EAH         LINE#         16
  C:61EFH         LINE#         17
  -------         ENDPROC       TPSTATE
  -------         PROC          SPISTAR
  C:61E1H         LINE#         20
  C:61E1H         LINE#         21
  C:61E1H         LINE#         22
  C:61E3H         LINE#         23
  C:61E5H         LINE#         24
  C:61E7H         LINE#         25
  C:61E9H         LINE#         26
  -------         ENDPROC       SPISTAR
  -------         PROC          _WRITECHARTO7843
  D:0007H         SYMBOL        num
  -------         DO            
  D:0006H         SYMBOL        count
  -------         ENDDO         
  C:6166H         LINE#         28
  C:6166H         LINE#         29
  C:6166H         LINE#         30
  C:6168H         LINE#         31
  C:616AH         LINE#         32
  C:616AH         LINE#         33
  C:616AH         LINE#         34
  C:616EH         LINE#         35
  C:6170H         LINE#         36
  C:6175H         LINE#         37
  C:617AH         LINE#         38
  C:617FH         LINE#         39
  -------         ENDPROC       _WRITECHARTO7843
  -------         PROC          READFROMCHARFROM7843
  -------         DO            
  D:0005H         SYMBOL        count
  D:0006H         SYMBOL        Num
  -------         ENDDO         
  C:60CFH         LINE#         42
  C:60CFH         LINE#         43
BL51 BANKED LINKER/LOCATER V6.22                                                      10/31/2017  16:00:21  PAGE 22


  C:60CFH         LINE#         44
  C:60D1H         LINE#         45
  C:60D3H         LINE#         46
  C:60D3H         LINE#         47
  C:60D3H         LINE#         48
  C:60DAH         LINE#         49
  C:60DFH         LINE#         50
  C:60E4H         LINE#         51
  C:60E7H         LINE#         52
  C:60E7H         LINE#         53
  C:60EBH         LINE#         54
  C:60EBH         LINE#         56
  C:60F0H         LINE#         58
  C:60F0H         LINE#         59
  -------         ENDPROC       READFROMCHARFROM7843
  -------         PROC          _ADS_READ_AD
  D:0007H         SYMBOL        CMD
  -------         DO            
  D:0006H         SYMBOL        l
  -------         ENDDO         
  C:6180H         LINE#         62
  C:6180H         LINE#         63
  C:6180H         LINE#         65
  C:6182H         LINE#         66
  C:6185H         LINE#         67
  C:618BH         LINE#         68
  C:6191H         LINE#         69
  C:6194H         LINE#         70
  C:6196H         LINE#         71
  C:6196H         LINE#         72
  -------         ENDPROC       _ADS_READ_AD
  -------         PROC          _ADS_READ_XY
  D:0001H         SYMBOL        xy
  -------         DO            
  D:0002H         SYMBOL        i
  X:007AH         SYMBOL        j
  X:007CH         SYMBOL        buf
  X:009AH         SYMBOL        sum
  X:009CH         SYMBOL        temp
  -------         ENDDO         
  C:4D1BH         LINE#         78
  C:4D1DH         LINE#         79
  C:4D1DH         LINE#         82
  C:4D24H         LINE#         84
  C:4D26H         LINE#         85
  C:4D26H         LINE#         86
  C:4D45H         LINE#         87
  C:4D50H         LINE#         88
  C:4D53H         LINE#         89
  C:4D53H         LINE#         90
  C:4D73H         LINE#         91
  C:4D73H         LINE#         92
  C:4DA5H         LINE#         93
  C:4DA5H         LINE#         94
  C:4DADH         LINE#         95
  C:4DDFH         LINE#         96
  C:4E03H         LINE#         97
BL51 BANKED LINKER/LOCATER V6.22                                                      10/31/2017  16:00:21  PAGE 23


  C:4E03H         LINE#         98
  C:4E17H         LINE#         99
  C:4E25H         LINE#         100
  C:4E2CH         LINE#         101
  C:4E5CH         LINE#         102
  C:4E71H         LINE#         103
  C:4E71H         LINE#         104
  -------         ENDPROC       _ADS_READ_XY
  -------         PROC          _READ_ADS
  X:00E4H         SYMBOL        x
  X:00E7H         SYMBOL        y
  -------         DO            
  X:00EAH         SYMBOL        xtemp
  D:0006H         SYMBOL        ytemp
  -------         ENDDO         
  C:5EB8H         LINE#         107
  C:5EC3H         LINE#         108
  C:5EC3H         LINE#         110
  C:5ED0H         LINE#         111
  C:5ED5H         LINE#         112
  C:5EEFH         LINE#         113
  C:5F07H         LINE#         114
  C:5F18H         LINE#         115
  C:5F1AH         LINE#         116
  -------         ENDPROC       _READ_ADS
  -------         PROC          _READ_ADS2
  X:00BFH         SYMBOL        x
  X:00C2H         SYMBOL        y
  -------         DO            
  X:00C5H         SYMBOL        x1
  X:00C7H         SYMBOL        y1
  X:00C9H         SYMBOL        x2
  X:00CBH         SYMBOL        y2
  D:0007H         SYMBOL        flag
  -------         ENDDO         
  C:50E8H         LINE#         121
  C:50F3H         LINE#         122
  C:50F3H         LINE#         126
  C:510AH         LINE#         127
  C:510FH         LINE#         128
  C:5126H         LINE#         129
  C:512BH         LINE#         130
  C:51C1H         LINE#         132
  C:51C1H         LINE#         133
  C:51EAH         LINE#         134
  C:5213H         LINE#         135
  C:5216H         LINE#         136
  C:5218H         LINE#         137
  -------         ENDPROC       _READ_ADS2
  -------         PROC          READ_TP_ONCE
  -------         DO            
  X:00F7H         SYMBOL        re
  X:00F8H         SYMBOL        x1
  X:00FAH         SYMBOL        y1
  -------         ENDDO         
  C:5D65H         LINE#         139
  C:5D65H         LINE#         140
BL51 BANKED LINKER/LOCATER V6.22                                                      10/31/2017  16:00:21  PAGE 24


  C:5D65H         LINE#         141
  C:5D6AH         LINE#         143
  C:5D70H         LINE#         144
  C:5D70H         LINE#         145
  C:5D8AH         LINE#         146
  C:5D91H         LINE#         147
  C:5DABH         LINE#         148
  C:5DD3H         LINE#         149
  C:5DD3H         LINE#         150
  C:5DD8H         LINE#         151
  C:5DD8H         LINE#         152
  C:5DDAH         LINE#         153
  C:5DDFH         LINE#         154
  -------         ENDPROC       READ_TP_ONCE
  -------         PROC          _DROW_TOUCH_POINT
  X:00FCH         SYMBOL        x
  X:00FEH         SYMBOL        y
  C:5219H         LINE#         156
  C:5227H         LINE#         157
  C:5227H         LINE#         158
  C:5230H         LINE#         159
  C:525AH         LINE#         160
  C:528EH         LINE#         161
  C:52ADH         LINE#         162
  C:52CCH         LINE#         163
  C:52EBH         LINE#         164
  C:530AH         LINE#         165
  -------         ENDPROC       _DROW_TOUCH_POINT
  -------         PROC          _TP_DRAW_BIG_POINT
  X:0100H         SYMBOL        x
  X:0102H         SYMBOL        y
  D:0002H         SYMBOL        color
  C:5DE0H         LINE#         170
  C:5DEEH         LINE#         171
  C:5DEEH         LINE#         172
  C:5DF8H         LINE#         174
  C:5E03H         LINE#         175
  C:5E1CH         LINE#         176
  C:5E35H         LINE#         177
  -------         ENDPROC       _TP_DRAW_BIG_POINT
  -------         PROC          CONVERT_POS
  -------         DO            
  D:0006H         SYMBOL        temp
  X:0108H         SYMBOL        l
  -------         ENDDO         
  C:4FAFH         LINE#         181
  C:4FAFH         LINE#         182
  C:4FAFH         LINE#         186
  C:4FB4H         LINE#         188
  C:4FD0H         LINE#         189
  C:4FD0H         LINE#         190
  C:4FD6H         LINE#         191
  C:5041H         LINE#         192
  C:50ACH         LINE#         193
  C:50ACH         LINE#         195
  C:50B4H         LINE#         196
  C:50C1H         LINE#         197
BL51 BANKED LINKER/LOCATER V6.22                                                      10/31/2017  16:00:21  PAGE 25


  C:50C7H         LINE#         198
  C:50E2H         LINE#         204
  C:50E7H         LINE#         205
  -------         ENDPROC       CONVERT_POS
  -------         PROC          TOUCH_ADJUST
  -------         DO            
  X:0000H         SYMBOL        vx1
  X:0004H         SYMBOL        vx2
  X:0008H         SYMBOL        vy1
  X:000CH         SYMBOL        vy2
  X:0010H         SYMBOL        chx1
  X:0012H         SYMBOL        chx2
  X:0014H         SYMBOL        chy1
  X:0016H         SYMBOL        chy2
  X:0018H         SYMBOL        lx
  X:001AH         SYMBOL        ly
  X:001CH         SYMBOL        p
  X:003CH         SYMBOL        cnt
  -------         ENDDO         
  C:2331H         LINE#         210
  C:2331H         LINE#         211
  C:2331H         LINE#         216
  C:2336H         LINE#         217
  C:2337H         LINE#         218
  C:233FH         LINE#         219
  C:2347H         LINE#         220
  C:234CH         LINE#         221
  C:2354H         LINE#         222
  C:2354H         LINE#         223
  C:2357H         LINE#         224
  C:2357H         LINE#         225
  C:2357H         LINE#         226
  C:235AH         LINE#         227
  C:235AH         LINE#         228
  C:2360H         LINE#         229
  C:2360H         LINE#         230
  C:2380H         LINE#         231
  C:239CH         LINE#         232
  C:23A2H         LINE#         233
  C:23A2H         LINE#         234
  C:23B4H         LINE#         235
  C:23B4H         LINE#         236
  C:23B4H         LINE#         237
  C:23BBH         LINE#         238
  C:23BEH         LINE#         239
  C:23BEH         LINE#         240
  C:23BEH         LINE#         241
  C:23D0H         LINE#         242
  C:23D3H         LINE#         243
  C:23D3H         LINE#         244
  C:23DAH         LINE#         245
  C:23DDH         LINE#         246
  C:23DDH         LINE#         247
  C:23DDH         LINE#         248
  C:23EFH         LINE#         249
  C:23F2H         LINE#         250
  C:23F2H         LINE#         251
BL51 BANKED LINKER/LOCATER V6.22                                                      10/31/2017  16:00:21  PAGE 26


  C:23F9H         LINE#         252
  C:23FCH         LINE#         253
  C:23FCH         LINE#         254
  C:23FCH         LINE#         255
  C:2418H         LINE#         256
  C:241BH         LINE#         257
  C:241BH         LINE#         258
  C:2422H         LINE#         259
  C:2425H         LINE#         260
  C:2425H         LINE#         261
  C:2425H         LINE#         262
  C:24E4H         LINE#         263
  C:258CH         LINE#         264
  C:2634H         LINE#         265
  C:26DCH         LINE#         267
  C:279BH         LINE#         268
  C:2843H         LINE#         269
  C:28EBH         LINE#         270
  C:2993H         LINE#         273
  C:2AD1H         LINE#         274
  C:2AD1H         LINE#         275
  C:2AD6H         LINE#         276
  C:2ADDH         LINE#         277
  C:2AE8H         LINE#         278
  C:2AEBH         LINE#         279
  C:2AEBH         LINE#         280
  C:2B51H         LINE#         281
  C:2B93H         LINE#         284
  C:2B9AH         LINE#         285
  C:2BA1H         LINE#         286
  C:2BA9H         LINE#         306
  C:2BB9H         LINE#         307
  C:2C14H         LINE#         308
  C:2C2BH         LINE#         309
  C:2C87H         LINE#         310
  C:2C9EH         LINE#         311
  C:2CFAH         LINE#         312
  C:2D11H         LINE#         313
  C:2D6DH         LINE#         315
  C:2D84H         LINE#         316
  C:2DA4H         LINE#         317
  C:2DBBH         LINE#         318
  C:2DDBH         LINE#         319
  C:2DDEH         LINE#         321
  C:2DE5H         LINE#         323
  C:2DE5H         LINE#         324
  C:2DE5H         LINE#         325
  C:2DE5H         LINE#         326
  -------         ENDPROC       TOUCH_ADJUST
  -------         ENDMOD        TOUCH

  -------         MODULE        LCD
  C:0000H         SYMBOL        _ICE_DUMMY_
  D:0090H         PUBLIC        P1
  D:00A0H         PUBLIC        P2
  D:00B0H         PUBLIC        P3
  C:61BCH         PUBLIC        _LCD_WR_REG
BL51 BANKED LINKER/LOCATER V6.22                                                      10/31/2017  16:00:21  PAGE 27


  C:5CE4H         PUBLIC        _LCD_Clear
  B:00B0H.3       PUBLIC        LCD_RESET
  C:614BH         PUBLIC        LCD_Reset
  C:6130H         PUBLIC        _LCD_WR_DATA_16Bit
  B:00B0H.2       PUBLIC        LCD_BL
  C:4405H         PUBLIC        LCD_Init
  B:0090H.3       PUBLIC        LCD_CS
  B:0090H.0       PUBLIC        LCD_RD
  C:6034H         PUBLIC        _LCD_DrawPoint
  C:5E54H         PUBLIC        _LCD_SetWindows
  C:5F64H         PUBLIC        LCD_SetParam
  C:61D6H         PUBLIC        LCD_WriteRAM_Prepare
  C:61C9H         PUBLIC        _LCD_WR_DATA
  B:0090H.2       PUBLIC        LCD_RS
  B:0090H.1       PUBLIC        LCD_WR
  C:61B2H         PUBLIC        _LCD_WriteReg
  C:6111H         PUBLIC        _LCD_SetCursor
  X:009EH         PUBLIC        POINT_COLOR
  X:00A0H         PUBLIC        BACK_COLOR
  X:00A2H         PUBLIC        lcddev
  -------         PROC          _LCD_WR_REG
  D:0006H         SYMBOL        Reg
  C:61BCH         LINE#         62
  C:61BCH         LINE#         63
  C:61BCH         LINE#         64
  C:61BEH         LINE#         65
  C:61C0H         LINE#         67
  C:61C2H         LINE#         72
  C:61C4H         LINE#         73
  C:61C6H         LINE#         74
  C:61C8H         LINE#         75
  -------         ENDPROC       _LCD_WR_REG
  -------         PROC          _LCD_WR_DATA
  D:0006H         SYMBOL        Data
  C:61C9H         LINE#         86
  C:61C9H         LINE#         87
  C:61C9H         LINE#         88
  C:61CBH         LINE#         89
  C:61CDH         LINE#         91
  C:61CFH         LINE#         96
  C:61D1H         LINE#         97
  C:61D3H         LINE#         98
  C:61D5H         LINE#         99
  -------         ENDPROC       _LCD_WR_DATA
  -------         PROC          _LCD_WR_DATA_16BIT
  D:0004H         SYMBOL        Data
  C:6130H         LINE#         110
  C:6134H         LINE#         111
  C:6134H         LINE#         112
  C:6136H         LINE#         113
  C:6138H         LINE#         115
  C:613CH         LINE#         116
  C:613EH         LINE#         117
  C:6140H         LINE#         118
  C:6144H         LINE#         119
  C:6146H         LINE#         120
  C:6148H         LINE#         127
BL51 BANKED LINKER/LOCATER V6.22                                                      10/31/2017  16:00:21  PAGE 28


  C:614AH         LINE#         128
  -------         ENDPROC       _LCD_WR_DATA_16BIT
  C:61AEH         SYMBOL        L?0022
  -------         PROC          L?0021
  -------         ENDPROC       L?0021
  C:61AEH         SYMBOL        L?0022
  -------         PROC          _LCD_WRITEREG
  D:0006H         SYMBOL        LCD_Reg
  D:0004H         SYMBOL        LCD_RegValue
  C:61B2H         LINE#         140
  C:61B2H         LINE#         141
  C:61B2H         LINE#         142
  C:61B5H         LINE#         143
  -------         ENDPROC       _LCD_WRITEREG
  -------         PROC          LCD_WRITERAM_PREPARE
  C:61D6H         LINE#         156
  C:61D6H         LINE#         157
  C:61D6H         LINE#         158
  -------         ENDPROC       LCD_WRITERAM_PREPARE
  -------         PROC          _LCD_CLEAR
  X:0104H         SYMBOL        Color
  -------         DO            
  X:0106H         SYMBOL        i
  D:0002H         SYMBOL        j
  -------         ENDDO         
  C:5CE4H         LINE#         171
  C:5CECH         LINE#         172
  C:5CECH         LINE#         174
  C:5D16H         LINE#         175
  C:5D32H         LINE#         176
  C:5D32H         LINE#         177
  C:5D42H         LINE#         178
  C:5D42H         LINE#         179
  C:5D4DH         LINE#         180
  C:5D54H         LINE#         182
  C:5D64H         LINE#         183
  -------         ENDPROC       _LCD_CLEAR
  -------         PROC          _LCD_DRAWPOINT
  D:0002H         SYMBOL        x
  D:0082H         SYMBOL        y
  C:6034H         LINE#         194
  C:603CH         LINE#         195
  C:603CH         LINE#         196
  C:6053H         LINE#         197
  -------         ENDPROC       _LCD_DRAWPOINT
  -------         PROC          LCD_RESET
  C:614BH         LINE#         209
  C:614BH         LINE#         210
  C:614BH         LINE#         211
  C:614DH         LINE#         212
  C:6154H         LINE#         213
  C:6156H         LINE#         214
  C:615DH         LINE#         215
  C:615FH         LINE#         216
  -------         ENDPROC       LCD_RESET
  -------         PROC          LCD_INIT
  C:4405H         LINE#         228
BL51 BANKED LINKER/LOCATER V6.22                                                      10/31/2017  16:00:21  PAGE 29


  C:4405H         LINE#         229
  C:4405H         LINE#         230
  C:4408H         LINE#         231
  C:440AH         LINE#         235
  C:4415H         LINE#         236
  C:441EH         LINE#         237
  C:4427H         LINE#         238
  C:442FH         LINE#         239
  C:4436H         LINE#         240
  C:443EH         LINE#         241
  C:4446H         LINE#         242
  C:444EH         LINE#         243
  C:4456H         LINE#         244
  C:445DH         LINE#         245
  C:4463H         LINE#         246
  C:446BH         LINE#         247
  C:4473H         LINE#         248
  C:447BH         LINE#         249
  C:4483H         LINE#         250
  C:448BH         LINE#         252
  C:4492H         LINE#         253
  C:4498H         LINE#         254
  C:449EH         LINE#         255
  C:44A6H         LINE#         256
  C:44AEH         LINE#         257
  C:44B6H         LINE#         258
  C:44BEH         LINE#         259
  C:44C5H         LINE#         260
  C:44CDH         LINE#         261
  C:44D5H         LINE#         262
  C:44DBH         LINE#         263
  C:44E3H         LINE#         264
  C:44EAH         LINE#         265
  C:44F2H         LINE#         266
  C:44FAH         LINE#         267
  C:4502H         LINE#         268
  C:4508H         LINE#         269
  C:450EH         LINE#         270
  C:4516H         LINE#         271
  C:451EH         LINE#         272
  C:4526H         LINE#         273
  C:452EH         LINE#         274
  C:4534H         LINE#         275
  C:453CH         LINE#         276
  C:4544H         LINE#         277
  C:454CH         LINE#         279
  C:4554H         LINE#         280
  C:455CH         LINE#         281
  C:4564H         LINE#         282
  C:456CH         LINE#         285
  C:4574H         LINE#         287
  C:457CH         LINE#         288
  C:4584H         LINE#         289
  C:458CH         LINE#         290
  C:4592H         LINE#         291
  C:459DH         LINE#         292
  C:45A4H         LINE#         293
BL51 BANKED LINKER/LOCATER V6.22                                                      10/31/2017  16:00:21  PAGE 30


  C:45AFH         LINE#         294
  C:45B6H         LINE#         295
  C:45C1H         LINE#         296
  C:45C8H         LINE#         298
  C:45D3H         LINE#         300
  C:45DCH         LINE#         302
  C:45E5H         LINE#         303
  C:45ECH         LINE#         304
  C:45F7H         LINE#         307
  C:45FAH         LINE#         308
  C:45FCH         LINE#         309
  -------         ENDPROC       LCD_INIT
  -------         PROC          _LCD_SETWINDOWS
  X:0072H         SYMBOL        xStar
  X:0074H         SYMBOL        yStar
  D:0002H         SYMBOL        xEnd
  X:0078H         SYMBOL        yEnd
  C:5E54H         LINE#         316
  C:5E62H         LINE#         317
  C:5E62H         LINE#         319
  C:5E6AH         LINE#         320
  C:5E72H         LINE#         321
  C:5E7DH         LINE#         322
  C:5E89H         LINE#         323
  C:5E8FH         LINE#         324
  C:5E9BH         LINE#         325
  C:5EA9H         LINE#         326
  C:5EB5H         LINE#         328
  -------         ENDPROC       _LCD_SETWINDOWS
  -------         PROC          _LCD_SETCURSOR
  D:0002H         SYMBOL        Xpos
  D:0082H         SYMBOL        Ypos
  C:6111H         LINE#         337
  C:6119H         LINE#         338
  C:6119H         LINE#         339
  -------         ENDPROC       _LCD_SETCURSOR
  -------         PROC          LCD_SETPARAM
  C:5F64H         LINE#         344
  C:5F64H         LINE#         345
  C:5F64H         LINE#         346
  C:5F6DH         LINE#         348
  C:5F73H         LINE#         349
  C:5F7BH         LINE#         350
  C:5F82H         LINE#         351
  C:5F8BH         LINE#         352
  C:5F92H         LINE#         353
  -------         ENDPROC       LCD_SETPARAM
  -------         ENDMOD        LCD

  -------         MODULE        ?C?FPADD
  C:2DEDH         PUBLIC        ?C?FPADD
  C:2DE9H         PUBLIC        ?C?FPSUB
  -------         ENDMOD        ?C?FPADD

  -------         MODULE        ?C?FPMUL
  C:2EDEH         PUBLIC        ?C?FPMUL
  -------         ENDMOD        ?C?FPMUL
BL51 BANKED LINKER/LOCATER V6.22                                                      10/31/2017  16:00:21  PAGE 31



  -------         MODULE        ?C?FPDIV
  C:2FE7H         PUBLIC        ?C?FPDIV
  -------         ENDMOD        ?C?FPDIV

  -------         MODULE        ?C?FPCMP
  C:3086H         PUBLIC        ?C?FPCMP
  C:3084H         PUBLIC        ?C?FPCMP3
  -------         ENDMOD        ?C?FPCMP

  -------         MODULE        ?C?FCAST
  C:3107H         PUBLIC        ?C?FCASTC
  C:3102H         PUBLIC        ?C?FCASTI
  C:30FDH         PUBLIC        ?C?FCASTL
  -------         ENDMOD        ?C?FCAST

  -------         MODULE        ?C?CASTF
  C:313BH         PUBLIC        ?C?CASTF
  -------         ENDMOD        ?C?CASTF

  -------         MODULE        ?C?CLDPTR
  C:31BCH         PUBLIC        ?C?CLDPTR
  -------         ENDMOD        ?C?CLDPTR

  -------         MODULE        ?C?CLDOPTR
  C:31D5H         PUBLIC        ?C?CLDOPTR
  -------         ENDMOD        ?C?CLDOPTR

  -------         MODULE        ?C?UIDIV
  C:3202H         PUBLIC        ?C?UIDIV
  -------         ENDMOD        ?C?UIDIV

  -------         MODULE        ?C?IILDX
  C:3257H         PUBLIC        ?C?IILDX
  -------         ENDMOD        ?C?IILDX

  -------         MODULE        ?C?ILDIX
  C:326DH         PUBLIC        ?C?ILDIX
  -------         ENDMOD        ?C?ILDIX

  -------         MODULE        ?C?ISTPTR
  C:3283H         PUBLIC        ?C?ISTPTR
  -------         ENDMOD        ?C?ISTPTR

  -------         MODULE        ?C?LMUL
  C:32A2H         PUBLIC        ?C?LMUL
  -------         ENDMOD        ?C?LMUL

  -------         MODULE        ?C?ULDIV
  C:332DH         PUBLIC        ?C?ULDIV
  -------         ENDMOD        ?C?ULDIV

  -------         MODULE        ?C?LNEG
  C:33BFH         PUBLIC        ?C?LNEG
  -------         ENDMOD        ?C?LNEG

  -------         MODULE        ?C?ULCMP
BL51 BANKED LINKER/LOCATER V6.22                                                      10/31/2017  16:00:21  PAGE 32


  C:33CDH         PUBLIC        ?C?ULCMP
  -------         ENDMOD        ?C?ULCMP

  -------         MODULE        ?C?LSTXDATA
  C:33DEH         PUBLIC        ?C?LSTXDATA
  -------         ENDMOD        ?C?LSTXDATA

  -------         MODULE        ?C?LSTKXDATA
  C:33EAH         PUBLIC        ?C?LSTKXDATA
  -------         ENDMOD        ?C?LSTKXDATA

  -------         MODULE        ?C?OFFXADD
  C:341BH         PUBLIC        ?C?OFFXADD
  -------         ENDMOD        ?C?OFFXADD

  -------         MODULE        STRLEN
  C:6197H         PUBLIC        _STRLEN
  -------         ENDMOD        STRLEN

Program Size: data=9.0 xdata=265 code=25072
LINK/LOCATE RUN COMPLETE.  0 WARNING(S),  0 ERROR(S)
